:020000020000FC
:100000000C9424000C947A080C947A080C947A08C6
:100010000C947A080C947A080C947A080C947A0858
:100020000C947A080C947A080C947A080C947A0848
:100030000C947A080C947A080C947A080C947A0838
:100040000C947A080C947A0809E102BB00E007BB23
:1000500000E001BB04E00EBF0FE50DBF07E109B9E9
:10006000539A549A0E944B08809902C0C4D6D9D79B
:100070000E944A084DD26FEFD3D14CD0FBCFE3950D
:10008000C8953196002009F0089550E0DDC1F9E0EF
:10009000EEEBF6DF091679F4F3DF081669F4F0DF0A
:1000A000071659F43196C895002D3196C895F02D54
:1000B000E02F09950895319631963396EACF90EF67
:1000C00080EF21E0088184D1513011F41AD0F7CFAC
:1000D000702F17D00D3091F0952E088179D10D3009
:1000E00069F0951639F4982F872F702F0AD0239531
:1000F000233099F708816CD1951609F0089501D045
:10010000F9CFD81529F4C71519F454E09DC1089505
:1001100021970895D0E0CFEF01EC702E00E0802E03
:10012000088156D1523009F494C0F2D1A16001C0C7
:10013000AE7F3DB7383010F458E086C1C0DF7D3067
:10014000B9F0092D023031F49F708F707F7042D268
:1001500020D0EFCF9F758F757F75213029F4092D41
:10016000033011F407D0E5CF92DF7D3009F0089518
:10017000A16008957154763212F055E065C175564C
:10018000A0FF11F406D00895F0E0E72F708101D0B0
:100190000895F3E0E62F70836A95633F10F456E00C
:1001A00053C108956395603012F057E04DC1F3E0FC
:1001B000E62F7081089520E2A1D120E29FD120E2B4
:1001C0009DD120E29BD1392F92D120E297D1382FB7
:1001D0008ED120E293D1372F8AD120E28FD108959A
:1001E00020E28CD120E28AD13E2F81D120E286D13B
:1001F00008955BE029C1D0E0CFEFFF24EE247727FC
:10020000BF7D0881CA95E3940D3041F0E1D05230B2
:1002100039F0B0625130A9F3F394F3CF0F2D089564
:10022000B5FF7395EECF54E00FC152E00DC19F7042
:100230008F707F70CFD10895D0E0CFEFE030A9F379
:1002400008810083319721970D30C1F75E2E6F2E04
:100250000895D1DF743068F6062D033021F4052DA2
:10026000033F09F452C0D0E0CFEF772788279927C2
:10027000C715CAF20881ACD0523029F4982F872FC5
:10028000702F2197F5CFD3DFA72EF62DE52DB77F61
:10029000BF7E992788277727BB243196F33011F446
:1002A000E43F59F0008194D0543039F0523089F74E
:1002B000B394782F892F902FF0CF0B2D033029F096
:1002C000B394782F892F90E0F8CFB4FD02C0B061CD
:1002D000E0CFADDFA71691F118F4B860DF2ECE2E77
:1002E000F33021F4E43F11F4B3FF0FC0B3FF08C0B3
:1002F0007A1508F442C0F33019F4E43F09F43DC024
:10030000F33039F6E43F29F6089575DF003009F43B
:100310000895D0E0CFEFF62DE52DF23019F4E0305E
:1003200009F409C008810083319721970D30A9F79E
:100330005E2E6F2E089502E0502F86C03197DF2F7A
:10034000CE2FD23019F4C03009F46DCF0881219737
:100350000D30B9F70E2F0C1B500E08F46394D230F9
:1003600011F4C03029F00881008321973197F7CF2D
:1003700042DF003009F06DCF08953DDF003039F1E4
:10038000062D023021F4052D00500E15A0F2F62D99
:10039000E52DDF2FCE2FCE19D0400C2F502E0D2F54
:1003A000602EFD1519F4EC1509F405C000810883D1
:1003B00021963196F6CFD0E0CFEFFD2DEC2D319781
:1003C000088100830D3019F031972197F9CF0895F6
:1003D0005527102F1D3009F416C01F75103009F471
:1003E00002C01C3011F451E0089510310AF4089550
:1003F0001B350AF00895103412F053E008951A31B5
:100400000AF452E0089554E00895CF3F19F427E02C
:1004100075D00AC0212F81D0C3951DE0188304C078
:100420002EE36CD0D0E0CFEF7DD0183071F318837D
:100430001D3049F0C23C19F427E060D0F5CFCA95D1
:10044000212F6BD0F1CF089563D0503021F4F6E026
:10045000E8EE6CD042C0513021F4F7E0E0E166D024
:100460003CC0523021F4F7E0EEE460D036C05330A7
:1004700021F4F7E0E0E75AD030C0543021F4F7E03F
:10048000E2EB54D02AC0553021F4F7E0E4EE4ED030
:1004900024C0563021F4F8E0E8E148D01EC05730BF
:1004A00021F4F8E0EAE542D018C0583021F4F8E031
:1004B000EAEB3CD012C0593021F4F9E0EAE136D041
:1004C0000CC05A3021F4F9E0E2E530D006C05B30D0
:1004D00021F4F9E0EAE82AD000C00FE504E00EBFFD
:1004E0000FE50DBF6FEFA0E0B0E012D0C3CD57D045
:1004F000242F04D0232F02D00895202F5D9BFECF00
:1005000066D6B6FF03C05F9BFECFBF7B2CB90895B4
:100510002DE0F4DF2AE0F2DF08952D3011F4F8DF4A
:100520000895ECCF5F9BFECF1CB10895C8950020C5
:1005300021F0202DE3DF3196F9CF0895F7DFE8DFD2
:10054000089530DE07E007174AF001E0703019F037
:10055000000F7A95FBCF702F1CDE08955AE074DFF0
:10056000903039F0905D292FC9DF803011F420E3FD
:10057000C5DF803019F0805D282FC0DF705D272F28
:10058000BDDF089599278827745610F09395FCCF06
:100590007C597A5010F08395FCCF765F0895432FF5
:1005A0004695469546954695405D4A3308F0495F25
:1005B0003F70305D3A3308F0395F089546FD475F7C
:1005C0004F7036FD375F3F70440F440F440F440FA8
:1005D000342B08959330B2F4923032F0863092F496
:1005E000853012F0763072F4882321F00AE0700F23
:1005F0008A9581F7992309F4089504E68894700F89
:100600009A95C0F751E020CF83DF82DFF6E0E4E186
:1006100095DF08952020202020204154544F42414E
:100620005349432076657273696F6E203136332DDE
:10063000303231313135432E204E6F7420666F7267
:1006400020636F6D6D65726369616C207573652ED3
:100650000A0D202020202020436F7079726967687E
:1006600074203230303220627920526963686172BE
:10067000642043617070656C7320616C6C207269DA
:10068000676874732072657365727665642E0A0DEF
:10069000202020202020687474703A2F2F70726FF1
:1006A0006A656374732E63617070656C732E6F720C
:1006B000672020202020202070726F6A6563747389
:1006C0004063617070656C732E6F72670A0D000075
:1006D00046726565202070616765733A00002020CE
:1006E00063686172733A00004572726F7220303A2B
:1006F00020556E6B6E6F776E20636F6D6D616E64EB
:10070000206F72206F70657261746F722E2000000E
:100710004572726F7220313A20456E636F756E7448
:100720006572656420612076616C7565207468610E
:1007300074206973206E6F74206265747765656ECE
:10074000203020616E64203235352E200000457245
:10075000726F7220323A2050726F6772616D206D35
:10076000656D6F72792069732066756C6C2E000060
:100770004572726F7220333A20456E636F756E74E6
:10078000657265642061206368617261637465727B
:100790002074686174206973206E6F742061207208
:1007A00065636F676E697A656420747970652E2061
:1007B00000004572726F7220343A28696E74657257
:1007C0006E616C206572726F72202D62756666654F
:1007D00072206C696D697420657863656564656411
:1007E000292000004572726F7220353A20496E61EF
:1007F0007070726F70726961746520766172696180
:10080000626C65206E616D6520656E636F756E74D8
:10081000657265642E2000004572726F7220363A50
:10082000204461746120737461636B207075736818
:10083000206572726F72202D746F6F206D616E79FA
:1008400020617267756D656E7473206F6E206F6EB8
:1008500065206C696E652E2000004572726F7220F3
:10086000373A204461746120737461636B20706F48
:1008700070206572726F722E0A0D202020202020B9
:1008800020202046756E6374696F6E2074726965EE
:100890006420746F2075736520612076616C7565C6
:1008A000207468617420776173206E6F74206176A4
:1008B00061696C61626C652E00004572726F722016
:1008C000383A204D616368696E6520737461636BAB
:1008D000206572726F720A0D2020202020202020B7
:1008E0002046756E6374696F6E7320616E642F6F3E
:1008F000722063616C6C73206E6573746564207420
:100900006F6F20646565706C79206F7220746F6FF3
:1009100020636F6D706C657800004572726F722095
:10092000393A20474F544F206F7220474F5355425A
:100930002064657374696E6174696F6E206C696E92
:100940006520776173206E6F7420666F756E642EFC
:1009500000004572726F7220413A205370656369DE
:10096000666965642062697420706F736974696F69
:100970006E2072616E6765206F6620302E2E3720E4
:10098000657863656564656400004572726F722006
:10099000423A204C696E65206E756D626572206802
:1009A0006173206D6F7265207468616E2074687267
:1009B0006565206E756D6572616C732000004C4931
:1009C0005320C70553495A20D3054E4557204A089E
:1009D00050500B203A0650500D2041065052494EBF
:1009E000E70550525820EE0550524220200750573C
:1009F0004D387006505745207A0650574F208606CE
:100A0000454D49541307501A1D20F60550501D201E
:100A1000FF05464F52209D064E4558541006501C67
:100A20001E20190650501E20890650501C206A06B0
:100A300050494620930650544F209F0650500420A2
:100A4000A30652554E201108454E4420A106414EA2
:100A5000442048064C5352204F064C534C20540619
:100A6000504F52205906584F5220600644554D5061
:100A70005D08474F544FD506474F5355D906524549
:100A80005455DC065448454E99064B4559201807E5
:100A900041434F20250653415645E2064C4F414401
:100AA000FB065045454B2B06504F4B4532064F44F5
:100AB0004120E0074F444220E4074F444320E80729
:100AC0004F444420EC074F504120D0074F50422064
:100AD000D4074F504320D8074F504420DC07494EDD
:100AE0004120F007494E4220F307494E4320F707C3
:100AF000494E4420FA07534241202C0743424120EB
:100B00003307534242203B074342422042075342AD
:100B100043204A0743424320510753424420590788
:100B20004342442060075344412068074344412026
:100B30006F07534442207707434442207E075344C3
:100B400043208607434443208D07534444209507A0
:100B5000434444209C0749424120A4074942422083
:100B6000AF0749424320BA0749424420C5074144E0
:100B70004320FE0744454C417B08445352459C08A2
:100B80004453434F96084453444590080000C0DC4A
:100B9000F3E0E3EFF61511F4E51521F02081BDDC5B
:100BA0003197F8CFB5DCB4DCF6E0E0EDBFDC752DB5
:100BB000962D70509240EDDA792FE4DCD1DCF6E02E
:100BC000EEEDB4DCEFDADEDCCBDCA2DC0895AE7F48
:100BD000B0DAE8DAD7DCC4DC9BDC0895A9DA24E2D9
:100BE0008DDCE0DA372F83DC93DC0895AE7FA1DA69
:100BF000D9DA072FD7DAF0E0E72F00830895A2FFB4
:100C000040C0AE7F96DACEDAA72ECCDA872FCADACA
:100C1000B72EF0E0E72F8083A062A860AA7F089536
:100C2000F0E0EB2D00810A1519F003950083A06117
:100C300008957EDAB7DA072FB5DA701719F077273B
:100C4000A8DA08957FEFA5DA089572DA70E0459B7F
:100C500071E09FDA08956CDAA5DAE72FF0E0708191
:100C600098DA089565DA9EDA072F9CDAF0E0E02F33
:100C7000708308955DDA96DA072F94DA700F89DAB7
:100C8000089556DA8FDA072F8DDA701B82DA08950D
:100C90004FDA88DA072F86DA70237BDA089548DA8C
:100CA00081DA769576DA089543DA7CDA770F71DAAD
:100CB00008953EDA77DA072F75DA702B6ADA08952D
:100CC00037DA70DA072F6EDA702763DA089571E089
:100CD00060DA08952DDA66DA072F64DA70171EC01D
:100CE00027DA01E80FBD0EBD8D9A5CDA00E00BBD7E
:100CF0007ABD08951DDA03E80FBD01E00EBDBD9A6F
:100D000051DA072F4FDA7BBD0ABD089500E00FBD11
:100D100008950EDA47DA072F45DA071770E0BAF6BA
:100D2000B1F237DA089504DA3DDA772309F0A260E8
:100D300008950DB70E5F0DBF0895A4600895F8D90A
:100D40000895B26008954881DCD9388137DC732F6B
:100D500020DAD7D9EDD90895EBD924DA472FF3E07B
:100D6000E3EF0AC0F61511F45E16E8F400810D30C9
:100D700011F03197F7CF3197772788279927F61504
:100D800011F45E1680F4008123DB523029F4982F91
:100D9000872F702F3197F3CF9F708F707F701ADC81
:100DA000471701F7089559E04FCBD6DFDF2FCE2F3D
:100DB0000895D2DFA06C0895B2FF02C0B16008951B
:100DC000B26008956FEF752DE4D9762DE2D9D3E0A6
:100DD000CFEFEFEFF1E00881E199FECFFFBBEEBB73
:100DE0000DBBE29AE19AD23011F4C03019F031977C
:100DF0002197F1CF0895D3E0CFEFEFEFF1E0E19944
:100E0000FECFFFBBEEBBE09A0DB30883D23011F4E6
:100E1000C03019F031972197F2CF6DEFC3D9672E0B
:100E2000C1D9572E089584D9BDD9272F67DB0895DE
:100E30005F9BFECF7CB1733009F4B260AAD90895EC
:100E400077D9B0D908E020E3771F08F421E356DB17
:100E50000A95C9F75DDB08956BD973DBA3D90BB392
:100E6000072B02BB089564D96CDB9CD970950BB33A
:100E7000072302BB08955CD964DB94D908B3072B20
:100E800002BB089555D95DDB8DD9709508B3072352
:100E900002BB08954DD955DB85D905B3072B02BB9D
:100EA000089546D94EDB7ED9709505B3072302BB62
:100EB00008953ED946DB76D902B3072B02BB0895CD
:100EC00037D93FDB6FD9709502B3072302BB089572
:100ED0002FD937DB67D90AB3072B0ABB089528D966
:100EE00030DB60D970950AB307230ABB089520D977
:100EF00028DB58D907B3072B07BB089519D921DB85
:100F000051D9709507B3072307BB089511D919DB91
:100F100049D904B3072B04BB08950AD912DB42D97F
:100F2000709504B3072304BB089502D90ADB3AD9AC
:100F300001B3072B01BB0895FBD803DB33D97095B0
:100F400001B307230ABB0895F3D8FBDA2BD909B301
:100F5000072370E0002309F471E01BD90895E8D855
:100F6000F0DA20D906B3072370E0002309F471E01A
:100F700010D90895DDD8E5DA15D903B3072370E059
:100F8000002309F471E005D90895D2D8DADA0AD934
:100F900000B3072370E0002309F471E0FAD8089544
:100FA000C7D800D97BBB0895C3D8FCD878BB0895B7
:100FB000BFD8F8D875BB0895BBD8F4D872BB0895D4
:100FC000B7D8F0D87ABB0895B3D8ECD877BB0895DA
:100FD000AFD8E8D874BB0895ABD8E4D871BB0895F6
:100FE00079B3D7D8089576B37C7FD3D8089573B3F7
:100FF000D0D8089570B37C7FCCD8089570E0C9D85C
:1010000097D8D0D87F71706E77B906ED06B936994A
:10101000FECF75B1BED80895427265616B200A0D8E
:101020000000D3E0C3EF6FEFA160D1D0A5FF03C0F4
:10103000CC2EDD2EAF7DA4FF03C0DD2DCC2DAF7EE9
:10104000A6FF03C0EC2EFD2EAF7BA7FF04C0DF2F51
:10105000CE2FB460AF77B0FF03C0DF2DCE2DBA7FA7
:10106000B1FF04C043D0D62DC52DBD7FD61511F4D8
:101070005C1678F40881ACD9A1FF04C0543011F09B
:101080002197D1CFAD7F523011F42197CCCF51D8D9
:10109000CACF0895B9DA03E0602E03EF502EF62D83
:1010A000E52D6FEFA0E0B0E000E0F23011F4E030A9
:1010B00019F000833197F9CF0895F3E0E3EFF230B0
:1010C00011F4E03041F0308112DA20E217DA20E248
:1010D00015DA3197F4CF1CDA1BDA362D08DA20E264
:1010E0000DDA352D04DA14DA13DA0895F0E1E8E1C7
:1010F0001DDA089518951CD855D8992788275527A3
:101100000027772361F09A958A955A954A95F1F7C9
:101110000A95E1F7D1F7C1F7B1F77A95F2CF0895C3
:1011200007D840D8172F88940BD0089501D83AD803
:10113000172F089405D0089527D0712F2AD8089525
:1011400001B3077E01BB02B3086102BB99E0839B38
:10115000FECF949A8C9810F094988C9A93988B9ACE
:101160002FD08B98939A2CD08399F8CF18F0949A1B
:101170008C9802C094988C9A839BFECF8C98949AFA
:10118000111F9A9521F7089501B3077E01BB02B3A1
:10119000086102BB99E08399FECF8894849B06C0C6
:1011A000089493988B9A8499FECF04C093988B9A55
:1011B000849BFECF8B98939A111F9A9561F708959F
:1011C00030E540E54A95F1F73A95D9F708955F9BE8
:1011D00009C00CB1033111F4B06404C00CB1033088
:0611E00009F4B26008955D
:00000001FF
